:10000000F9C0000013C1000011C100000FC10000C1
:100010000DC100000BC1000009C1000007C10000B4
:1000200005C1000003C1000001C100000C944E1284
:10003000FDC00000FBC00000F9C0000065C7000063
:10004000F5C00000F3C00000F1C0000099C100003D
:10005000EDC00000EBC00000E9C00000E7C00000F8
:10006000E5C00000E3C00000E1C00000DFC0000008
:10007000DDC0000018034100560052004900530043
:10008000500020006D006B004900490000000C0387
:10009000410054004D0045004C00000004030904D9
:1000A00012011001FF000010EB0304210002010205
:1000B00003014000410142430309000A000A000B0A
:1000C000000C000D000D000E000F001000100012BB
:1000D0000013001300140016001600180019001A6F
:1000E000001C001D001F0020002200230025002707
:1000F0000029002B002E0030003200340037003A77
:10010000003D004000430046004A004E00520055AA
:10011000005A005E00630068006D00730078007E86
:100120000084008B0091009900A000A900B100B9E3
:1001300000C300CC00D600E100EC00F70004011180
:10014000011E012D013B014B015B016C017D019101
:1001500001A501BA01CF01E601FE01160231024CF0
:10016000026A028802A802CA02ED02110338036083
:10017000038B03B803E70318044B048104B904F5A7
:100180000434057505B90501064E069D06EF0648BF
:1001900007A30704086508D0084009B6092B0AAB75
:1001A0000A300BC30B510CEE0C8F0D400EF60EAF48
:1001B0000F681047111412F512ED13E214F015F93F
:1001C000161B185C19911AE51B251D831E0320AB15
:1001D00021302332250F27F128F82A1A2D492FA183
:1001E000311434A1364539173C1A3F34426045DF9B
:1001F00048704C0011241FBECFEFD2E0DEBFCDBF50
:1002000011E0A0E0B1E0E8E7F8E202C005900D924D
:10021000A23AB107D9F721E0A2EAB1E001C01D92EC
:10022000A53BB207E1F744D00C943A14E9CE95B15E
:100230009F71982B95B9089584B7877F84BF88E113
:100240000FB6F89480936000109260000FBE90E0AB
:1002500080E80FB6F89480936100909361000FBE20
:1002600084B1806E84B985B18F7185B90C943F12C9
:1002700080ECDDCF80E4DBCF42E360E882E00E94E7
:10028000A711882311F080E801C080E4D0CF8EB39D
:10029000843069F4D3D182E08093E9008091E80052
:1002A00082FF05C080ECC3DF88D080E8C0CF08950E
:1002B000C3DF7BD080E4BBDF7894489B02C090E032
:1002C00001C090E285B18F7D892B85B9E0DF0E9466
:1002D0000514F3CF00C0D9011C92292F33272230F7
:1002E000310541F02330310561F02130310509F449
:1002F00039C03DC082E08C93E0E2F0E08EE191E015
:100300003AC099278130910589F01CF4892B39F086
:100310002EC08230910589F0039749F515C0ECE9AC
:10032000F0E0E491F0E08CE990E025C0EEE8F0E048
:10033000E491F0E08EE890E01EC0E4E7F0E0E491A4
:10034000F0E084E790E017C0E0910001F0E082E384
:1003500090E090930F0180930E0182E08C9380E0F7
:1003600091E009C0E2E1F0E080EA90E004C0E0E062
:10037000F0E080E090E0DA018D939C93CF01089546
:1003800078941F920F920FB60F9211248F938AB513
:10039000882321F08AB581508ABD01C015BC8F9198
:1003A0000F900FBE0F901F9018958BE987BD82E0CC
:1003B00084BD80936E0027D1D5C50F931F93CF9333
:1003C000DF931F92CDB7DEB71091F10084E68ABDAE
:1003D00085E085BD143109F4C4C000F51A3009F474
:1003E000A7C068F4143038F4123008F050C011304F
:1003F00009F0CFC02FC0163009F0CBC073C0113147
:1004000009F4AAC020F4103109F0C3C0A3C012310E
:1004100009F4AAC0133109F0BCC0A0C0193109F415
:10042000A8C060F4163109F49CC008F497C01731D5
:1004300009F49FC0183109F0ACC098C01D3109F40F
:100440009BC008F493C0103509F49AC0113509F027
:10045000A0C094C08091E8008B778093E80082E090
:100460008093E9008091EC0081608093EC00109310
:10047000F1001092F1008AE08093F10040E050E03A
:100480006AE070E087E991E00E947E0F98C00091D9
:10049000F100123011F46091F1008091E8008B7747
:1004A0008093E80082E08093E9008091EC00816015
:1004B0008093EC001093F100802F6983C0D0698194
:1004C000123039F481FF0CC01092F100802FC7D098
:1004D00076C080FF05C01092F100802FB8D06DC0AB
:1004E00080EC6BC040E050E064E070E086EA91E0B0
:1004F0000E941A108091E8008B778093E80082E0D8
:100500008093E9008091EC0081608093EC00809101
:10051000A6019091A701A091A801B091A901B7FFF0
:1005200003C081E08093A50186E08093F1000FC0B5
:100530008091E8008B778093E80082E08093E90067
:100540008091EC0081608093EC001093F100109298
:10055000F10035C055D438C01FD436C0812FC2D069
:1005600033C0812FFBD130C0CAD32EC0812F94D28B
:100570002BC0812FECD228C030D326C03AD724C05C
:1005800068D722C08091E8008B778093E8000E94B2
:10059000DA118091F2008034A9F38091E8008B7722
:1005A0008093E80082E08093E9008091EC00816014
:1005B0008093EC001093F10089EC8093F10080911E
:1005C000E8008E778093E80015BC0E94DA1182E083
:1005D0008093E9008091EC008E7F8093EC000F9077
:1005E000DF91CF911F910F910895EEE3F1E090819B
:1005F000891739F0339691E0EC35F907C1F7E0E05F
:10060000F0E0CF010895CF93DF9380E090E00E9467
:100610002014D82F81E090E00E942014C82FDF3FE3
:1006200021F08EE9E2DFFC01D283CF3F21F088E99F
:10063000DCDFFC01C283DF91CF9108950895D5DFFF
:10064000009719F0FC018181089580E00895CDDFC5
:10065000009719F0FC018281089580E008951F93AE
:10066000CF93DF931F92CDB7DEB7182F6983BDDF1D
:100670006981009789F0FC0162831E3919F480E0DA
:1006800090E004C0183941F481E090E00F90DF91D0
:10069000CF911F910C9428140F90DF91CF911F914F
:1006A000089590915C01992329F08EBD0DB407FE49
:1006B000FDCF0895BEC490915C01992331F08EBDA9
:1006C0000DB407FEFDCF8EB50895B3C480915C01D3
:1006D000882331F01EBC0DB407FEFDCF8EB5089502
:1006E00080E0A7C45F926F927F928F929F92AF92A9
:1006F000BF92CF92DF92EF92FF920F931F93CF930F
:10070000DF93CDB7DEB7CA50D1400FB6F894DEBF45
:100710000FBECDBF182F40E050E069E070E0CE0181
:1007200001960E94CC0F6A8179817A836983613056
:1007300081E0780788F08091E8008B778093E8006B
:1007400082E08093E9008091EC0081608093EC006E
:100750001093F10080ECE4C040E050E0CE010A9636
:100760000E94CC0F89819A810A968F739927892BD1
:1007700039F48091E8008B778093E8000E94DA11C9
:100780008091E8008B778093E80082E08093E90015
:100790008091EC0081608093EC00133111F4988417
:1007A00001C099848090A6017090A701C12CD12C22
:1007B0005E01EAE0AE0EB11CE12CF12C88E0682E5F
:1007C0005524539477C0F50101915F019B8180917D
:1007D000A501882369F0C65FDE4F9883CA50D140D7
:1007E0007BD41092A501C65FDE4F9881CA50D140DC
:1007F0008D81C65FDE4F9883CA50D14052DF809111
:10080000A7014FDF8091A6014CDF802F4ADFC65F32
:10081000DE4F9881CA50D140133119F42D8126251D
:100820002D83E114F10479F4091569F08F81C0FE7C
:1008300004C0133111F4886001C0877F8F83E0907A
:10084000A601F090A70190FD11C0E114F10421F47C
:1008500093FD02C0997F92600F812C81492DB701D1
:10086000892F43D481112DC0E12CF12CC0FC02C092
:100870001531E9F48091A6019091A701A091A801FA
:10088000B091A9010196A11DB11D8093A60190937D
:10089000A701A093A801B093A901133141F4AA279D
:1008A000BB27892B8A2B8B2B11F45092A501FFEFCC
:1008B000CF1ADF0A89819A81C816D90608F483CF36
:1008C00080E09B8197FF2AC08E81EBDE872DE9DED9
:1008D000882DE7DE80E0E5DE8B8185FF06C0E11430
:1008E000F10419F48F7C80618B830F812C81492D59
:1008F000B7018B81FAD3133189F44091A60150914D
:10090000A7016091A8017091A90166277727452B5F
:10091000462B472B19F491E09093A5011093F10019
:100920008093F1008091E8008E778093E800C65FA5
:10093000DE4F0FB6F894DEBF0FBECDBFDF91CF9173
:100940001F910F91FF90EF90DF90CF90BF90AF90ED
:100950009F908F907F906F905F900895DF92EF92BD
:10096000FF920F931F93CF93DF9300D01F92CDB7C9
:10097000DEB7F82E40E050E063E070E0CE01019673
:100980000E94CC0F89819A8199838A838091E800A3
:100990008B778093E80082E08093E9008091EC00FF
:1009A00081608093EC00F092F1001092F10000E081
:1009B00010E098E0E92EDD24D39449C08091A50190
:1009C000882319F089D31092A5018B816ADE80916A
:1009D000A70167DE8091A60164DE78DE8093F100D6
:1009E0008091E80085FD07C08091E8008E778093B4
:1009F000E8000E94DA1184E1F81203C08B818E2591
:100A00008B8300FD03C086E1F8121FC04091A60150
:100A10005091A7016091A8017091A9014F5F5F4FAC
:100A20006F4F7F4F4093A6015093A7016093A80199
:100A30007093A90186E1F81641F066277727452BC8
:100A4000462B472B11F4D092A5010F5F1F4F298130
:100A50003A810217130708F4B1CF1092F100909178
:100A6000E8008091E8008E778093E80095FD09C04A
:100A70000E94DA118091E8008E778093E8000E944E
:100A8000DA110F900F900F90DF91CF911F910F917E
:100A9000FF90EF90DF900895BF92CF92DF92EF9298
:100AA000FF920F931F93CF93DF93CDB7DEB72997B4
:100AB0000FB6F894DEBF0FBECDBFB82E40E050E0B9
:100AC00065E070E0CE0101960E94CC0F9091E800A5
:100AD0009B779093E80082E08093E9009091EC008E
:100AE00091609093EC008E010E5F1F4F7E0186E0B7
:100AF000E80EF11C6701F80181918F01DCDDF7013F
:100B000081937F010C151D05B1F7B092F100109291
:100B1000F1008981FE01E80FF11D85818093F100CC
:100B20001092F1008091E8008E778093E80029967A
:100B30000FB6F894DEBF0FBECDBFDF91CF911F91EE
:100B40000F91FF90EF90DF90CF90BF900895DF92CC
:100B5000EF92FF920F931F93CF93DF9300D000D0BB
:100B6000CDB7DEB7D82E40E050E064E070E0CE01B3
:100B700001960E94CC0F9091E8009B779093E8003B
:100B800082E08093E9009091EC0091609093EC00FA
:100B90008E010F5F1F4F7E0185E0E80EF11CF8010A
:100BA00081918F017EDD0E151F05C9F7D092F100EE
:100BB0001092F1001092F1008091E8008E778093FE
:100BC000E8000F900F900F900F90DF91CF911F9141
:100BD0000F91FF90EF90DF900895FF920F931F9376
:100BE000CF93DF93CDB7DEB7C250D1400FB6F894A4
:100BF000DEBF0FBECDBF40E050E063E070E0CE014D
:100C000001960E94CC0F69818E010C5F1F4F40E05E
:100C100050E070E0C8010E94CC0F8091E8008B7713
:100C20008093E80082E08093E9008091EC0081608D
:100C30008093EC008DE18093F1001092F100F12C93
:100C40000BC08981F81628F4F801EF0DF11D8081A1
:100C500001C080E026DDF3948B81F81690F310E05C
:100C60001CC08981F81650F4E4E0F0E0EC0FFD1FA1
:100C7000EF0DF11DF39480811EDD01C027DD80930F
:100C8000F1008091E80085FD07C08091E8008E7733
:100C90008093E8000E94DA111F5F8A81181708F319
:100CA0001092F1009091E8008091E8008E77809397
:100CB000E80095FD09C00E94DA118091E8008E7766
:100CC0008093E8000E94DA11CE5FDE4F0FB6F894F1
:100CD000DEBF0FBECDBFDF91CF911F910F91FF906F
:100CE000089506C0EFE9FFE03197F1F700C000007A
:100CF000882321F09AB581509111F4CF0895EF9295
:100D0000FF920F931F93CF93DF9300D000D000D0BA
:100D1000CDB7DEB740E050E066E070E0CE0101966E
:100D20000E94CC0F8091E8008B778093E80082E0EE
:100D30008093E9008091EC0081608093EC008E014B
:100D40000D5F1F4F7E0187E0E80EF11CF8018191D5
:100D50008F01A7DC0E151F05C9F78A81811104C018
:100D60008981BFDF80E001C099D192E19093F100C9
:100D70008093F1008091E8008E778093E8002696BA
:100D80000FB6F894DEBF0FBECDBFDF91CF911F919C
:100D90000F91FF90EF9008950F931F93CF93DF93E0
:100DA00000D0CDB7DEB740E050E062E070E0CE01A9
:100DB00001960E94CC0F08EE10E0F80180818B773D
:100DC000808382E08093E900ECEEF0E08081816036
:100DD0008083898186DF80E055D1D8D08A8181DF08
:100DE000E1EFF0E081E180831082F80180818E776D
:100DF00080830F900F90DF91CF911F910F910895F5
:100E0000CF92DF92EF92FF920F931F93CF93DF93D6
:100E1000CDB7DEB72F970FB6F894DEBF0FBECDBFAC
:100E200040E050E06BE070E0CE0101960E94CC0FF4
:100E30008091E8008B778093E80082E08093E9005E
:100E40008091EC0081608093EC001092A6011092DA
:100E5000A7011092A8011092A9018B8142DFC2D094
:100E600081E010D18A813DDF7E018CE0E80EF11C2B
:100E700023C08D8136DFF80181918F011CDCF601E2
:100E800081936F010E151F05A1F78F81882351F003
:100E9000EBE0F0E0EC0FFD1FE80FF11D90818E817B
:100EA000981302C080E017C080E0ECD08A8119DF7F
:100EB00081E0E8D08A8115DF8C81982F91509C8346
:100EC000882341F08AB5882329F08E01085F1F4FDF
:100ED0006701CFCF80EC90E19093F1008093F10017
:100EE0008091E8008E778093E8002F960FB6F894F3
:100EF000DEBF0FBECDBFDF91CF911F910F91FF904D
:100F0000EF90DF90CF9008951F920F920FB60F923F
:100F100011248F93199908C08091A30187FF02C003
:100F20002A9A19C02A9817C08091A301880F80932C
:100F3000A3018091A20181508093A201811104C07C
:100F40001092810082E086BB1B9B05C08091A301AB
:100F500081608093A301199A8F910F900FBE0F901B
:100F60001F9018953E9A10926F0010928500109273
:100F7000840081E090E0909389008093880080E471
:100F80008093800089E080938100089580915C01C6
:100F9000882349F084B1897F84B985B1867F85B97A
:100FA0001CBC1DBC089584B1897F84B985B1867F3E
:100FB00085B9D8CF92E090936F001092850010927F
:100FC0008400E82FF0E0EE0FFF1FE555FF4F8591FD
:100FD00094919093890080938800109280001092E1
:100FE0008100089588E933DB8730D0F491E0909355
:100FF0005C01E82FF0E0EE54FF4FE491209A289A2C
:1010000084B1866084B923982B9A8DB5E6FF02C01F
:10101000816001C08E7F8DBD2098E065ECBD089594
:1010200010925C0194B1966094B995B1996095B9AC
:10103000C1CF8093A30188E08093A2018091A30196
:1010400087FF02C02A9A01C02A9810928500109248
:1010500084008AE0809381008091A201882319F0A6
:101060008AB58111F9CF109281008091A301089572
:1010700090915C01992329F08EBD0DB407FEFDCF40
:101080000895D7CF882339F0249A8EE9E0DA8111C8
:1010900003C02C9A089524982C98089580EFE8DFD7
:1010A00080E0E6DF80E0E4DF80915C01882331F0BE
:1010B0001EBC0DB407FEFDCF8EB502C080E0B9DFC7
:1010C00080FF03C08AB58111E9CF8AB5882311F06A
:1010D00080E0089581E808958DE4CADF80E0C8DFEC
:1010E0008091A801C5DF80E0C3CF0F931F93CF93FA
:1010F000DF93EB01142F8E77E82FF0E0E830F10555
:1011000069F134F4E230F10559F0349749F50BC038
:10111000E032F10541F0E034F10501F1709701F59D
:10112000822FDFDD1DC0802FA3DF8D2FA1DF8C2F4D
:101130009FDF80915C01882331F01EBC0DB407FE57
:10114000FDCF8EB502C080E074DF811303C08AB585
:101150008111E9CF8AB5882329F002C09FDF03C03F
:1011600080E001C080E894E69ABDDF91CF911F91A5
:101170000F9108959B01692F782F832F922F089547
:10118000CF93DF93CDB7DEB7C750D1400FB6F894F9
:10119000DEBF0FBECDBF40E050E067E070E0CE01A3
:1011A0008F5F9E4FF9D6CE5FDE4F688179818A814D
:1011B0009B81C250D140DEDFCE5FDE4F68837983F2
:1011C0008A839B83C250D140CA5FDE4F8881C6505C
:1011D000D140C95FDE4F9881C750D140CA5FDE4F12
:1011E0009883C650D140C95FDE4F8883C750D14035
:1011F0008091E8008B778093E80082E08093E9009B
:101200008091EC0081608093EC008091A401CA5F22
:10121000DE4F28813981C650D140811112C0CE5F86
:10122000DE4F688179818A819B81C250D140AE01B5
:101230004F5F5F4FE8D3882311F080E00EC083E05A
:101240000CC0A901BE016F5F7F4FCE5FDE4F88816A
:101250009981C250D140D1D5EECF90E59093F10065
:1012600095E09093F1008093F10081110BC0CA5F6B
:10127000DE4F68817981C650D14040E050E0CE0118
:1012800001963CD68091E8008E778093E800C95F94
:10129000DE4F0FB6F894DEBF0FBECDBFDF91CF910A
:1012A0000895AF92BF92CF92DF92EF92FF920F9389
:1012B0001F93CF93DF93CDB7DEB7C850D1400FB6A1
:1012C000F894DEBF0FBECDBF40E050E068E070E0B4
:1012D000CE01019661D66B817C818D819E814ADF32
:1012E0006B837C838D839E837F8168856F83788702
:1012F00040E050E0CE0109964FD68F81988509963F
:101300008F739927892B39F48091E8008B7780932C
:10131000E8000E94DA118091E8008B778093E80062
:1013200082E08093E9008091EC0081608093EC0082
:101330008091A40181112EC029812150EB80FC8075
:101340000D811E812630A0F430E0F901E359FE4FF3
:101350008081F901ED58FE4F9081F901E758FE4F69
:101360006081F901E158FE4F2081222359F103C029
:1013700066E293E28EE2AF80B88429E0C22ED12CDF
:10138000CC0EDD1E2A81482F892FB0D381110BC0CE
:1013900083E00AC04F815885BE01675F7F4F8B8114
:1013A0009C8157D5F3CF80E090E59093F10094E0D5
:1013B0009093F1008093F1008091E8008E77809304
:1013C000E80005C02985B801A70162D3DFCFC85F57
:1013D000DE4F0FB6F894DEBF0FBECDBFDF91CF91C9
:1013E0001F910F91FF90EF90DF90CF90BF90AF9043
:1013F0000895CF93DF931F92CDB7DEB740E050E062
:1014000061E070E0CE010196C7D58091E8008B774E
:101410008093E80082E08093E9008091EC00816095
:101420008093EC0089818093A40181E58093F10091
:101430008981813011F080E001C080EC8093F1005F
:101440008091E8008E778093E8000F90DF91CF9134
:101450000895CF93DF93CDB7DEB729970FB6F894F1
:10146000DEBF0FBECDBF8091F100843009F492C081
:1014700040F4823079F108F049C0813009F02BC185
:1014800009C0863009F48AC008F486C0873009F0A4
:1014900022C1CDC08091E8008B778093E80082E084
:1014A0008093E9008091EC0081608093EC00809152
:1014B000A401811102C01DD205C0823011F44FD4A5
:1014C00001C080E090E59093F10091E09093F100ED
:1014D0008927FAC09091E8009B779093E800809369
:1014E000E9008091EC0081608093EC008091A40180
:1014F000811102C045D201C075D480E58093F1000E
:1015000082E08093F1001092F100E0C040E050E0F2
:1015100065E070E0CE0101963FD56A817B818C81C8
:101520009D8128DE6A837B838C839D838091E80084
:101530008B778093E80082E08093E9008091EC0053
:1015400081608093EC008091A401E981811114C035
:10155000E150E83028F4F0E0EB59FE4F808101C003
:1015600080E04A815B816C817D8135D3882311F0D5
:1015700080E00BC083E009C0E13011F480E101C0DC
:1015800084E16A817B819DD4F1CF90E59093F10055
:1015900093E098C086DE9FC0F3DD9DC040E050E040
:1015A00061E070E0CE010196F7D48091E8008B777E
:1015B0008093E80082E08093E9008091EC008160F4
:1015C0008093EC008091A401811112C0E981E15067
:1015D000E23028F4F0E0EB57FE4F808101C088E74D
:1015E000BE016A5F7F4FD7D1882321F080E003C01E
:1015F00081E001C083E090E59093F10096E0909344
:10160000F1008093F100811161C08E819F81A885D6
:10161000B985CD01AA27BB278093F1008E819F81D8
:10162000A885B9858093F100892F99274DC08091B5
:10163000F100833029F128F4813041F0823081F5C6
:1016400016C0843011F1853059F524C08091F10025
:101650009091F1002091F1003091F10030936101FF
:1016600020936201909363018093640117C080917D
:10167000F1009091F10090935F01809360010EC0A2
:101680008091F10080935E0109C08091F100809308
:101690005D0104C08091F1008091F10080E001C003
:1016A00081E09091E8009B779093E80092E090931E
:1016B000E9009091EC0091609093EC0090E590939C
:1016C000F10097E09093F1008093F1008091E800A1
:1016D0008E778093E80029960FB6F894DEBF0FBE90
:1016E000CDBFDF91CF9108954D99FECF4D9BFECF99
:1016F0004D99FECF5B9A539A8091C9008F7E80935B
:10170000C9008091C90088608093C90081E08093FE
:10171000AA0108958091C80086FFFCCF8091C8007F
:1017200080648093C8008091C900877F8093C9003E
:101730008091C90080618093C90053985B98109292
:10174000AA0108958091AA018111E4DF80EC8093C1
:10175000C8001092C9001092CA008AB1877D8AB968
:101760008BB1837D8BB908958091AA018111D2DF5D
:101770008091C800806C8093C8001092C9001092BC
:10178000CA008AB1877D8AB98BB1837D8BB92498D1
:101790002C980895CF93DF931F92CDB7DEB7909129
:1017A000AA01911103C089839FDF89819091C800AC
:1017B00095FFFCCF9091C80090649093C8008093EF
:1017C000CE000F90DF91CF9108958091AA018111F1
:1017D000A1DF8091C80087FD03C08AB58111F9CFD0
:1017E0008091CE0008958091AA01811101C07CDF13
:1017F0008CE04D99FECF4D9BFECF4D99FECF815091
:10180000C1F708951092AA01249A2C988FE891E0CC
:101810000197F1F700C000008AB188628AB9529836
:1018200083E090E09093CD008093CC0088E080939B
:10183000C9008FE68093CA00D6DFD5CF1092AA01E7
:101840008AB188628AB952985B9A8FE891E00197D1
:10185000F1F700C0000083E090E09093CD0080930A
:10186000CC0088E08093C9008FE68093CA00BBDF7C
:10187000BACF1F93CF93DF9300D0CDB7DEB7182F29
:10188000862F79839A8386DF7981872F83DF812F63
:1018900081DF9A81892F0F900F90DF91CF911F9157
:1018A00079CF409161015091620160916301709123
:1018B0006401482BCB01BA01DCCF80E86BDF85DF08
:1018C0009AB5992321F081FFF8CF81E0089580E057
:1018D00008958BE65FDF8FE0E4DF80E25BDF75DF9A
:1018E0009AB5992321F087FDF8CF81E0089580E033
:1018F0000895BF92CF92DF92EF92FF920F931F93C2
:10190000CF93DF93CDB7DEB728970FB6F894DEBF3D
:101910000FBECDBF93DF81EC3DDF89E53BDF82EC7D
:1019200039DF82E037DF80EE35DF7E0189E0E80EC7
:10193000F11C8E010F5F1F4F88E0D82EB02EC12EF4
:10194000E7E8F1E0AB2DBC2D8D2D01900D928A952D
:10195000E1F7F70182917F011DDFE016F10681F7C3
:1019600028960FB6F894DEBF0FBECDBFDF91CF91A2
:101970001F910F91FF90EF90DF90CF90BF909DCF80
:101980009CDF81EC07DF80E005DF81E803DF1DDFFE
:101990008111F7CFD7CE1F93CF93DF93182FEB0191
:1019A000188219821A821B8294DF811101C026C01D
:1019B0008CE4F0DE8AE075DF812FECDE8CE4EADE79
:1019C0008BE06FDF81E0E6DE78DF8823B9F081DF2E
:1019D0008823A1F08BE6DEDE84E063DF80EADADED6
:1019E00082E0D8DE84E2D6DEF0DE8883EEDE898314
:1019F000ECDE8A839AB581E0911101C080E0DF912D
:101A0000CF911F910895CF92DF92EF92FF920F93A3
:101A10001F93CF93DF936B017C01EA01890159DFAA
:101A2000882361F18CE4B6DE8AE03BDF83E4B2DE3A
:101A300002301105C0F08BE6ADDEC701B60119DF3B
:101A400080EAA8DE802F8150A5DE84E2A3DE0C0FA1
:101A50001D1F02C0BADE8993C017D10759F08AB59D
:101A60008111F8CF07C08CE095DEC701B60101DF18
:101A7000ACDE88839AB581E0911101C080E0DF91EE
:101A8000CF911F910F91FF90EF90DF90CF9008952D
:101A90000F931F93CF93DF9300D000D0CDB7DEB765
:101AA000182F022F49835A836B837C8312DF88238C
:101AB00099F08CE46FDE8AE0F4DE812F6BDE8CE43B
:101AC00069DE49815A816B817C81CB01BA01D1DE0B
:101AD000802F60DE81E001C080E00F900F900F90BA
:101AE0000F90DF91CF911F910F9108952F923F9208
:101AF0004F925F926F927F928F929F92AF92BF921E
:101B0000CF92DF92EF92FF920F931F93CF93DF93C9
:101B1000782E662E842E922E17012801E60120FFD2
:101B200011C0D7DE811102C080E042C08CE432DEF9
:101B30008AE0B7DE862D2EDE8CE42CDE8BE0B1DE73
:101B400081E028DEA114B10419F491FC1FC02FC05C
:101B5000C0DE882349F38CE41DDE8AE0A2DE872DF7
:101B600019DE8BE617DEC201B10183DE80EA12DEE8
:101B70008A2D81500FDE84E60DDEAC0EBD1E02C044
:101B8000899108DECA15DB05D9F7DFCFA2DE8823ED
:101B900009F4CACF8CE4FEDD8AE083DE882DFADD0D
:101BA0008CE4F8DDC201B10164DE80E0F3DD81E0A8
:101BB000DF91CF911F910F91FF90EF90DF90CF9029
:101BC000BF90AF909F908F907F906F905F904F905D
:101BD0003F902F9008951F93CF93DF9300D000D0B4
:101BE000CDB7DEB7182F49835A836B837C8371DEB0
:101BF00049815A816B817C81882309F467C08CE418
:101C0000103429F4C7DD8AE04CDE80E440C049830B
:101C10005A836B837C83103309F040C0BBDD8AE0BC
:101C200040DE86E3B7DD8CE4B5DD8BE03ADE81E0B3
:101C3000B1DD4FDE882309F449C08CE4ABDD8AE0D6
:101C400030DE83E3A7DD8BE6A5DD49815A816B8118
:101C50007C81CB01BA010DDE80EA9CDD80915F01C1
:101C6000815098DD84E696DD10E003C080E092DDCF
:101C70001F5F212F30E080915F0190916001281754
:101C80003907A0F38CE486DD8AE00BDE80E382DD99
:101C90008CE480DD8BE005DE81E00FC07BDD8AE037
:101CA00000DE812F77DD8CE475DD49815A816B81FF
:101CB0007C81CB01BA01DDDD80E06CDD0F900F90FF
:101CC0000F900F90DF91CF911F91F7CD80E00F9093
:101CD0000F900F900F90DF91CF911F910895282FB3
:101CE000207330E0220F331F20693F6F8F70822BEB
:101CF00051CD1F93CF93DF931F92CDB7DEB7182F2F
:101D000088E6998347DD812F45DD89E643DD9981AA
:101D1000892F0F90DF91CF911F913CCD80E83ADD64
:101D200054DD9AB5992321F081FFF8CF81E0089521
:101D300080E0089580915D01282F207330E0220F0C
:101D4000331F20618F70822B25DD3FDD9AB59923EB
:101D500021F087FDEFCF81E0089580E00895BF92E4
:101D6000CF92DF92EF92FF920F931F93CF93DF9367
:101D7000CDB7DEB728970FB6F894DEBF0FBECDBF44
:101D800041DD82EC07DD82E005DD80EE03DD7E01D2
:101D900089E0E80EF11C8E010F5F1F4F58E0D52E31
:101DA000B02EC12EEFE8F1E0AB2DBC2D8D2D0190B2
:101DB0000D928A95E1F7F70182917F01EBDCE01645
:101DC000F10681F728960FB6F894DEBF0FBECDBF9F
:101DD000DF91CF911F910F91FF90EF90DF90CF9007
:101DE000BF909CCF9BDF80ECD5DC80E0D3DC80E82B
:101DF000D1DCEBDC8111F7CFB7CCEF92FF920F93E0
:101E00001F93CF93DF937C01EB018A0193DF88233B
:101E1000C1F080915E0163DF80E0BCDCC70169DF57
:101E20000C0F1D1F04C084E2B5DCCFDC8993C01702
:101E3000D10719F08AB58111F6CF9AB581E09111D9
:101E400001C080E0DF91CF911F910F91FF90EF9043
:101E50000895EF92FF920F931F93CF93DF937C012E
:101E60008B01EA0167DF811102C080E023C0C0FF5F
:101E700006C0F801EC0FFD1F8FEF80832196809143
:101E80005E012DDF8DE186DCC70133DF10C052DF3C
:101E9000882359F384E67EDCF80180817BDC84E6CC
:101EA00079DCF80181810E5F1F4F74DC2297209747
:101EB00071F781E0DF91CF911F910F91FF90EF902B
:101EC00008951F93CF93DF93182FEB0133DF8823FF
:101ED00081F080915E0103DF812F5CDCCE018160A7
:101EE00008DF80E657DC80E055DCDF91CF911F9161
:101EF00021CF80E0DF91CF911F910895BF92CF92C3
:101F0000DF92EF92FF920F931F93CF93DF937C01A9
:101F10008B01EA014FD2B82E811133C0209731F0E6
:101F200028813981021B130BE20EF31EC12CD12C28
:101F300023C08091E80085FD15C08091E8008E7770
:101F40008093E80062D4209749F0888199818C0DB4
:101F50009D1D9983888325E0B22E13C02BD2882340
:101F600059F00EC0F70181917F018093F10001507B
:101F70001109FFEFCF1ADF0A01151105D1F601C0D3
:101F8000B82E8B2DDF91CF911F910F91FF90EF9085
:101F9000DF90CF90BF900895BF92CF92DF92EF92E3
:101FA000FF920F931F93CF93DF937C018B01EA0184
:101FB00001D2B82E811133C0209731F028813981A8
:101FC000021B130BE20EF31EC12CD12C23C08091F7
:101FD000E80085FD15C08091E8008B778093E800CC
:101FE00014D4209749F0888199818C0D9D1D998387
:101FF000888345E0B42E13C0DDD1882359F00EC08C
:102000008091F100F70181937F0101501109FFEFE9
:10201000CF1ADF0A01151105D1F601C0B82E8B2D9C
:10202000DF91CF911F910F91FF90EF90DF90CF90B4
:10203000BF900895BF92CF92DF92EF92FF920F93DD
:102040001F93CF93DF936C018B017A01B3D1B82E2C
:1020500081113AC0E8012197CC0DDD1DE114F10496
:1020600039F0F70120813181021B130BC21BD30B06
:10207000C12CD12C24C08091E80085FD17C080912F
:10208000E8008B778093E800C0D3E114F10451F0AD
:10209000F701808191818C0D9D1D9183808355E096
:1020A000B52E12C087D1882351F00DC08091F10068
:1020B0008883219701501109FFEFCF1ADF0A01151C
:1020C0001105C9F601C0B82E8B2DDF91CF911F915C
:1020D0000F91FF90EF90DF90CF90BF9008952091E7
:1020E000B3013091B4012617370748F06115710527
:1020F00039F42091E8002E772093E80001C0B9015F
:102100009C0180E033C09EB3992309F444C095300C
:1021100009F443C09091E80093FD41C09091E8001C
:1021200092FD33C09091E80090FF20C08091F200B2
:1021300090E0F901821B930B05C021912093F100DF
:10214000615071099F01280F391F6115710519F040
:102150002031310590F381E02031310509F080E034
:102160009091E8009E779093E8009F0161157105BA
:1021700051F68111C8CF09C08EB3882361F0853034
:1021800061F08091E80083FD0AC08091E80082FF41
:10219000F3CF80E0089582E0089583E0089581E020
:1021A00008952091B3013091B4012617370748F004
:1021B0006115710539F42091E8002E772093E8002D
:1021C00001C0B9019C0180E034C09EB3992309F499
:1021D00045C0953009F444C09091E80093FD42C099
:1021E0009091E80092FD34C09091E80090FF21C0EA
:1021F0008091F20090E0F901821B930B06C02491BC
:102200002093F1003196615071099C012E0F3F1F00
:102210006115710519F02031310588F381E0203115
:10222000310509F080E09091E8009E779093E800F6
:102230009F016115710549F68111C7CF09C08EB3A1
:10224000882361F0853061F08091E80083FD0AC049
:102250008091E80082FFF3CF80E0089582E0089546
:1022600083E0089581E00895EF92FF920F931F930A
:10227000CF93DF938B012091B3013091B4012617E6
:10228000370748F06115710539F42091E8002E7781
:102290002093E80001C08901382F492F20E036C083
:1022A0008EB3882309F447C0853009F446C0809175
:1022B000E80083FD44C08091E80082FD36C0809133
:1022C000E80080FF23C0E090F200F12CC32FD42F50
:1022D000EC1AFD0A07C0CE01B3D28093F10021961B
:1022E00001501109CE018E0D9F1D0115110519F028
:1022F0008031910580F321E0409709F020E0809142
:10230000E8008E778093E8003C2F4D2F01151105D2
:1023100039F62111C5CF09C08EB3882361F085300D
:1023200061F08091E80083FD0AC08091E80082FF9F
:10233000F3CF80E005C082E003C083E001C081E00C
:10234000DF91CF911F910F91FF90EF9008958F70C3
:102350008093E900EBEEF0E0808181608083EDEE18
:10236000F0E010826093EC0040838091EE00881FC3
:102370008827881F08958091AD0187FD05C0809151
:10238000E80080FF0DC010C08091E80082FD04C00D
:102390008EB38111F9CF08958091E8008B7707C043
:1023A0008EB38111ECCF08958091E8008E778093F1
:1023B000E80008958091E4009091E50045E62091C1
:1023C000EC0020FD1EC022C02EB3222391F0253048
:1023D00091F02091EB0025FD10C02091E400309198
:1023E000E5002817390759F34150C90141F784E046
:1023F000089582E0089583E0089581E0089580E0E3
:1024000008952091E80020FFDFCFF9CF2091E80068
:1024100022FFDACFF4CF3CD03ED08091D8008F7726
:102420008093D8008091D80080688093D8008091F4
:10243000D8008F7D8093D80084E089BD86E089BD77
:1024400009B400FEFDCF1EBA1092AB0142E160E07C
:1024500080E07DDF8091E1008E7F8093E1008091BC
:10246000E20081608093E2008091E20088608093C6
:10247000E2008091E0008E7F8093E0000895E3E623
:10248000F0E080818E7F808381E08093AC01C3CFB8
:102490001092E20008951092E10008951F920F92A9
:1024A0000FB60F9211242F933F934F935F936F9327
:1024B0007F938F939F93AF93BF93EF93FF938091FD
:1024C000E10080FF17C08091E20080FF13C080917F
:1024D000E2008E7F8093E2008091E2008061809331
:1024E000E2008091D80080628093D80019BC1EBAA7
:1024F0000E943A018091E10084FF2FC08091E200A8
:1025000084FF2BC084E089BD86E089BD09B400FE4C
:10251000FDCF8091D8008F7D8093D8008091E1001D
:102520008F7E8093E1008091E2008F7E8093E200B5
:102530008091E20081608093E2008091AB0188236A
:1025400011F084E007C08091E30087FF02C083E0C0
:1025500001C081E08EBB0E9438018091E10083FFC1
:1025600021C08091E20083FF1DC08091E100877F40
:102570008093E10082E08EBB1092AB018091E1007C
:102580008E7F8093E1008091E2008E7F8093E20055
:102590008091E20080618093E20042E160E080E0AF
:1025A000D6DE32D1FF91EF91BF91AF919F918F9184
:1025B0007F916F915F914F913F912F910F900FBE3F
:1025C0000F901F9018951F93CF93DF9300D01F9209
:1025D000CDB7DEB7EDEAF1E08091F100819381E0C3
:1025E000E53BF807C9F710D18091E80083FFF7C0F9
:1025F0008091AD019091AE01953009F470C038F42E
:10260000913079F170F0933009F0E9C02AC0983028
:1026100009F4B7C0993009F4C6C0963009F0DFC09C
:1026200083C0803899F0823809F0D9C08091B10117
:102630009091B2018F7099278093E9009091EB00FF
:1026400095FB992790F91092E90001C090E08091E4
:10265000E800877F8093E8009093F1001092F100EA
:102660009BC0882319F0823009F0B9C08F71823085
:1026700009F0B5C08091AF0181112BC08091B101EB
:102680009091B2018F709927009709F4A8C08093A8
:10269000E9002091EB0020FF1CC02091AE01233007
:1026A00021F48091EB00806212C09091EB00906168
:1026B0009093EB0021E030E001C0220F8A95EAF709
:1026C0002093EA001092EA008091EB0088608093EA
:1026D000EB001092E9008091E800877F60C08111D3
:1026E0007EC08091AF019091B0018F779927182F0C
:1026F0009091E3009078982B9093E3008091E8000C
:10270000877F8093E80037DE8091E80080FFFCCF70
:102710008091E30080688093E300112311F083E04F
:1027200001C082E08EBB5BC08058823008F057C089
:102730009E012D5F3F4FAE014F5F5F4F6091B10132
:102740008091AF019091B0010E946A01BC01009795
:1027500009F445C08091E800877F8093E8002B81D1
:1027600089819A81211102C01CDD05C0213011F43C
:102770007BDD01C0B4DC8091E8008B778093E800BA
:102780002EC0803861F58091E800877F8093E80053
:102790008091AB018093F1008091E8008E77809367
:1027A000E800E9DD1CC081111AC09091AF019230A0
:1027B000B0F48091E800877F8093E8009093AB01AC
:1027C000DADD8091AB01811104C08091E30087FFC5
:1027D00002C084E001C081E08EBB0E943C01809178
:1027E000E80083FF0AC08091E800877F8093E800BB
:1027F0008091EB0080628093EB000F900F900F9020
:10280000DF91CF911F9108950895CF938EB38823C0
:10281000A9F08091E9008F709091EC0090FF02C0C8
:1028200090E801C090E0C92FC82B1092E900809178
:10283000E80083FDC8DECF70C093E900CF91089512
:10284000F999FECF92BD81BDF89A992780B5089578
:10285000262FF999FECF92BD81BDF89A019700B459
:10286000021639F01FBA20BD0FB6F894FA9AF99AF9
:082870000FBE0895F894FFCF9C
:102878001C033000300030003200300030003000DF
:102888003100320033003400350000000000090236
:102898002000010100C0320904000002FF0000000E
:1028A8000705820240000A0705020240000A80016B
:1028B800008101009001009101019201179401210A
:1028C8009803069E0301A10110A4030001323320DE
:1028D80000C001000140206830222A3218242C351B
:1028E8004C081A232333232323262636262626019B
:1028F800010100000138391289AB45CDD888FF1293
:1029080089AB45CDD888FF4156524953505F4D4B4E
:0229180032008B
:00000001FF
